:1000000030C03FC03EC03DC03CC03BC02AC139C02B
:1000100038C037C036C08CC1B7C133C032C031C060
:1000200030C02FC02EC0570D0A006D412020004760
:10003000656E657261746F723A2000570D0A006D2B
:10004000412020004C6F61643A20202020202000B5
:1000500064560D0A00566F6C746167653A20202063
:10006000000011241FBECFE5D4E0DEBFCDBF10E0FD
:10007000A0E6B0E001C01D92AD3AB107E1F75FD054
:10008000A1C3BECF8EB58B608EBD82EE94E09BBDCA
:100090008ABD80E189BF7894089587B3876087BB64
:1000A00088B3887F88BB0895CF93DF9382E064E0B4
:1000B00006D1BC0180E090E07FD223E333E343ED3F
:1000C00050E4E6D14DD2709363006093620081E00A
:1000D00064E0F5D09C012E5F3140C8E4D0E02C9F55
:1000E000C0012D9F900D3C9F900D112490936500B1
:1000F0008093640080E064E0E2D09C012F5F314097
:100100002C9FC0012D9F900D3C9F900D112490932A
:10011000670080936600DF91CF910895FC01CB01C9
:1001200024E630E0B901EAD26E9FC0016F9F900DC6
:100130007E9F900D1124B901CDD2862F0895EF92A4
:10014000FF920F931F93DF93CF93CDB7DEB72A971C
:100150000FB6F894DEBF0FBECDBF9FDF99D092DF00
:1001600083E390E036D1C09AC19AC2988E010F5FA6
:100170001F4F84E6E82EF12C97DF85E590E07BD1D8
:100180008091620090916300B8014AE050E0EBD2A8
:100190005FD180E590E06FD184E490E06CD18091F4
:1001A000660090916700B8014AE050E0DCD250D17F
:1001B0008FE390E060D18091660090916700B70175
:1001C0009DD22091620030916300629FC001639FC5
:1001D000900D729F900D1124B7017CD2862F90E074
:1001E000B8014AE050E0BFD233D18BE390E043D175
:1001F0008FE290E040D18091640090916500B80159
:100200004AE050E0B0D224D18AE290E034D180912B
:10021000640090916500B70171D220916200309125
:100220006300629FC001639F900D729F900D112427
:10023000B70150D2862F90E0B8014AE050E093D247
:1002400007D186E290E017D184E663D084E661D0DE
:1002500084E65FD084E65DD084E65BD084E659D046
:100260008BCF1F920F920FB60F9211248F939F93F3
:10027000809160009091610001969093610080935D
:1002800060009F918F910F900FBE0F901F90189557
:1002900080E487B983E086B9379A369A3699FECFDB
:1002A00084B195B1089597B18F71907E892B87B9EC
:1002B000369A3699FECF24B135B1C9010895BF925F
:1002C000CF92DF92EF92FF920F931F93D82EB62E0C
:1002D000CC24EE24FF2487010AC08D2DE4DFAC017D
:1002E00060E070E0E40EF51E061F171FC394CB14E8
:1002F000A0F32B2D30E040E050E0C801B70111D24F
:10030000C9011F910F91FF90EF90DF90CF90BF90A8
:100310000895882309F484E690E007C0E3ECF9E04F
:100320003197F1F700C000009F5F9817B8F3089568
:100330001F920F920FB60F9211242F938F939F93BA
:10034000EF93FF939BB18CB1E0918A00EF5FEF7167
:1003500020918B00E21741F09871E0938A00F0E061
:10036000E457FF4F808301C092E08091AC00892B5D
:100370008093AC00FF91EF919F918F912F910F90FF
:100380000FBE0F901F9018951F920F920FB60F92ED
:1003900011248F939F93EF93FF9390916800809126
:1003A0006900981761F0E0916900EF5FEF71E093E9
:1003B0006900F0E0E659FF4F80818CB901C0559883
:1003C000FF91EF919F918F910F900FBE0F901F9013
:1003D0001895109268001092690010928A0010928D
:1003E0008B0097FF03C022E02BB99F7790BD89B99E
:1003F00088E98AB986E880BD089590918A00809145
:100400008B00981781F0E0918B00EF5FEF71E09324
:100410008B00F0E0E457FF4F20818091AC001092F8
:10042000AC0030E002C020E031E0C90108959091B5
:1004300068009F5F9F71209169009217E1F3E92F97
:10044000F0E0E659FF4F808390936800559A089535
:10045000EF92FF92CF93DF93E82EE7017E01F92E12
:10046000E70101C0E4DF89918823E1F7DF91CF91B3
:10047000FF90EF900895CF93DF93EC0101C0D7DF99
:10048000FE01219684918823D1F7DF91CF910895C1
:100490000CD0E6C0DED040F0D5D030F021F45F3F84
:1004A00019F0C7C0511110C1CAC0EBD098F39923FD
:1004B000C9F35523B1F3951B550BBB27AA27621728
:1004C0007307840738F09F5F5F4F220F331F441F6D
:1004D000AA1FA9F333D00E2E3AF0E0E830D09150A5
:1004E0005040E695001CCAF729D0FE2F27D0660F92
:1004F000771F881FBB1F261737074807AB07B0E8D1
:1005000009F0BB0B802DBF01FF2793585F4F2AF0E6
:100510009E3F510568F08DC0D7C05F3FECF3983E19
:10052000DCF3869577956795B795F7959F5FC9F743
:10053000880F911D9695879597F90895E1E0660FCC
:10054000771F881FBB1F621773078407BA0720F045
:10055000621B730B840BBA0BEE1F88F7E0950895AE
:1005600098D088F09F5790F0B92F9927B751A0F0F5
:10057000D1F0660F771F881F991F1AF0BA95C9F737
:1005800012C0B13081F09FD0B1E008959CC0672FB8
:10059000782F8827B85F39F0B93FCCF386957795E7
:1005A0006795B395D9F73EF49095809570956195D0
:1005B0007F4F8F4F9F4F0895E89409C097FB3EF4FB
:1005C00090958095709561957F4F8F4F9F4F9923A0
:1005D000A9F0F92F96E9BB279395F695879577951E
:1005E0006795B795F111F8CFFAF4BB0F11F460FFDE
:1005F0001BC06F5F7F4F8F4F9F4F16C0882311F036
:1006000096E911C0772321F09EE8872F762F05C049
:10061000662371F096E8862F70E060E02AF09A95E4
:10062000660F771F881FDAF7880F9695879597F9D9
:10063000089597F99F6780E870E060E008959FEF64
:1006400080EC089500240A94161617061806090669
:10065000089500240A941216130614060506089538
:10066000092E0394000C11F4882352F0BB0F40F4C0
:10067000BF2B11F460FF04C06F5F7F4F8F4F9F4F00
:10068000089557FD9058440F551F59F05F3F71F082
:100690004795880F97FB991F61F09F3F79F08795E9
:1006A0000895121613061406551FF2CF4695F1DF72
:1006B00008C0161617061806991FF1CF8695710502
:1006C000610508940895E894BB2766277727CB0136
:1006D00097F90895AA1BBB1B51E107C0AA1FBB1FB6
:1006E000A617B70710F0A61BB70B881F991F5A95BE
:1006F000A9F780959095BC01CD01089597FB092E2F
:1007000007260AD077FD04D0E5DF06D000201AF4D2
:10071000709561957F4F0895F6F7909581959F4F5D
:100720000895A1E21A2EAA1BBB1BFD010DC0AA1F32
:10073000BB1FEE1FFF1FA217B307E407F50720F04A
:10074000A21BB30BE40BF50B661F771F881F991FC5
:100750001A9469F760957095809590959B01AC010E
:10076000BD01CF010895FB019F01E8944230BCF028
:100770004532ACF44A3029F497FB1EF490958195EC
:100780009F4F642F7727A6DF805D8A330CF0895D49
:100790008193CB010097A9F716F45DE25193108283
:1007A000C90100C0DC01FC01672F71917723E1F7DB
:1007B000329704C07C916D9370836291AE17BF072E
:0807C000C8F30895F894FFCF7F
:00000001FF
